:020000040000FA
:0400000000000528CF
:0800080008008B137D20A020ED
:10001000AB01051185100330A3005F20A020AA01C9
:10002000061C1528861C1D28102819302B060319BC
:10003000AB01AB0AB0202620102877204D20861374
:100040000617861606168615061563002B082B2044
:10005000AC00860008008207FF347F34BF34DF34F1
:10006000EF34F7347734B734D734E734FB347B34A8
:10007000BB34DB34EB34F3347334B334D334E33490
:100080006334A334C3344334833403340608AC00EC
:100090008609D2202C0886000800051585145F20EB
:1000A000051185105F20051585145F200511851049
:1000B0005F20051585145F20051185100800A30B2E
:1000C00065282C0886000330A300C830A0006430E7
:1000D00081000108031D6928A00B6728FF308600F6
:1000E00008003B30A1005F20A10B732808002B08FB
:1000F000A2007120A20B792808008B1383168113AC
:100100000117811201128111011581100110831252
:100110008B110B128B120B138D018C0183168D0129
:100120008C018312831662308F0083120030A0018D
:10013000AA01831600308500033086008312080070
:10014000861706178616061686150615080005304A
:10015000A8001E30A900A80BAB28A90BAB280800EB
:10016000A720061CB0280800A720861CB428080079
:100170002A1CBD2886172A10080086132A14080096
:10018000AA1CC5280617AA1008000613AA140800FE
:10019000A7008617D2208613D2208617D220A70B5D
:1001A000CB280800A801A901A80BD428A90BD428A2
:0201B000080045
:02400E00113F60
:02401000FC3F73
:00000001FF
